:020000040000FA
:0600000047EF0FF01200B3
:020006002C00CC
:06000800DEEF03F0120020
:02000E00C250DE
:08001000040B01E0010E1200D7
:0600180010EF04F01200DD
:02001E000100DF
:0C002000D81E0000000100009A00000043
:04002C008A8C938C9B
:10003000938E010EE66E55EC0FF0E55281AC07D0C1
:10004000939E010EE66E55EC0FF0E552938E120072
:100050008A9E939E939C010EE66E55EC0FF0E5523E
:10006000938E00000000000081AC06D00101400E1C
:10007000A46F400E03D002D0000E00D01200010E7B
:10008000E66E55EC0FF0E55281BE05D00101630E1E
:10009000A46F03D002D0000E00D012000101080EA0
:1000A0009B6F8A9E9A6B939E010EE66E55EC0FF045
:1000B000E552938C010EE66E55EC0FF0E552938EEF
:1000C000010EE66E55EC0FF0E55281BE05D0D7DF8C
:1000D000000902E0210E16D0FE0ED814D86E0101E0
:1000E0009A51E8249A6FFE0E9A159A6F81AC03D04C
:1000F000010E9A119A6F9B059B6F9B510008D3E3E9
:100100009A5100D01200D9CFE6FFE1CFD9FF01010B
:10011000080E9B6FFE0EDBCF9AF18A9E81BE06D041
:10012000AEDF000902E0FF0E27D021D09A37D8A019
:100130000ED0939E938C010EE66E55EC0FF0E552B7
:10014000938E010EE66E55EC0FF0E5520ED0939EA5
:100150008A9C939C010EE66E55EC0FF0E552938E4F
:10016000010EE66E55EC0FF0E55201019B0701010F
:100170009B51D4E1000E00D0E552E7CFD9FF120029
:100180008A9E939E938C010EE66E55EC0FF0E5521D
:10019000938E010EE66E55EC0FF0E5528A9C939C0F
:1001A000010EE66E55EC0FF0E55212008A9E939E0A
:1001B0008A9C939C010EE66E55EC0FF0E552938EEF
:1001C000010EE66E55EC0FF0E552938C010EE66ED3
:1001D00055EC0FF0E55212008A9C939C010EE66EDE
:1001E00055EC0FF0E5521200D9CFE6FFE1CFD9FF71
:1001F000FD0EDBCFE9FFFE0EDBCFEAFFEF5018E08C
:10020000FD0EDBCFE9FFDB2AFE0EDBCFEAFF01E3C9
:10021000DB2AEF50E66E77DFE552000903E0FF0EC0
:1002200009D005D015DF000902E0FF0E03D0E0D7AA
:10023000000E00D0E552E7CFD9FF1200D9CFE6FF7C
:10024000E1CFD9FF020EE126FC0EDBCFF3FFDB0688
:10025000F350000935E022DFDE6EDD6A010EDB506F
:10026000FF0B03E0FF0E2ED00BD0FD0EDBCFE9FF1E
:10027000DB2AFE0EDBCFEAFF01E3DB2ADFCFEFFF55
:10028000FC0EDB500EE1939E938C010EE66E55EC56
:100290000FF0E552938E010EE66E55EC0FF0E5522D
:1002A0000ED0939E8A9C939C010EE66E55EC0FF047
:1002B000E552938E010EE66E55EC0FF0E552C4D771
:1002C000000E00D0106E020EE15C02E2E16AE5521F
:1002D000E16E1050E552E7CFD9FF1200D9CFE6FF0B
:1002E000E1CFD9FF79DF640EE66EE66AE66AE66A78
:1002F00005EC06F0E552E552E552E552FE0EDBCF85
:10030000E6FF01DFE5520101A66FA2DE0101A66F43
:100310000A0EE66EF8DEE5520101A66F99DE0101D4
:10032000A66FE66AF0DEE5520101A66F91DE0101DB
:10033000A66F3CDF51DFFE0EDBCFE6FFE4DEE552C9
:100340000101A66F85DE0101A66FE66ADCDEE552DB
:100350000101A66F7DDE0101A66FE66AD4DEE552DB
:100360000101A66F75DE0101A66FE668CCDEE552DD
:100370000101A66F6DDE0101A66FE66AC4DEE552DB
:100380000101A66F65DE0101A66FE668BCDEE552DD
:100390000101A66F5DDE0101A66F08DF1DDFFE0E05
:1003A000DBCFE6FFB0DEE5520101A66F51DE0101B1
:1003B000A66F0D0EE66EA7DEE5520101A66F48DEC0
:1003C0000101A66FE6689FDEE5520101A66F40DEDF
:1003D0000101A66FEBDEE552E7CFD9FF1200D9CFBE
:1003E000E6FFE1CFD9FFF8DE640EE66EE66AE66A64
:1003F000E66A05EC06F0E552E552E552E552FE0EDE
:10040000DBCFE6FF80DEE55223DE0101A66F120E90
:10041000E66E79DEE5521CDE0101A66FFD0EDBCF34
:10042000E6FF71DEE55214DE0101A66FBFDEE55284
:10043000E7CFD9FF1200D9CFE6FFE1CFD9FFE652CF
:10044000CBDE640EE66EE66AE66AE66ADEDBE5525D
:10045000E552E552E552FCDD0101A66FFE0EDBCF51
:10046000E6FF51DEE5520101A66F640EE66EE66A14
:10047000E66AE66ACADBE552E552E552E552E8DD96
:100480000101A66FFD0EDBCFE6FF3DDEE552010167
:10049000A66F640EE66EE66AE66AE66AB6DBE552C9
:1004A000E552E552E552D4DD0101A66F7FDE640E10
:1004B000E66EE66AE66AE66AA8DBE552E552E552D0
:1004C000E5528ADEFE0EDB28E66E1DDEE5520101F6
:1004D000A66F640EE66EE66AE66AE66A96DBE552A9
:1004E000E552E552E552B4DD0101A66FD7DDDF6EBE
:1004F000640EE66EE66AE66AE66A87DBE552E55276
:10050000E552E55293DD52DEDF5000D0E552E55270
:10051000E7CFD9FF12000101A46B5EDED00EE66EBC
:10052000F2DDE5520101A46F93DD0101A66F8C0E8F
:10053000E66EE9DDE5520101A46F8ADD0101A66FD7
:10054000D6EF00F0D9CFE6FFE1CFD9FF0101A46BD0
:10055000CB6BCC6BCD6BCE6BFD0EDBCF06F0FE0E06
:10056000DBCF07F0030E061801E1075018E0020E7A
:10057000061801E1075010E0010E061801E10750CE
:1005800008E0065001E1075001E00BD0200EC46FD7
:1005900008D0400EC46F05D0600EC46F02D0C46B8B
:1005A00000D00C0EC56FC66BC551126E136A800E5B
:1005B000C425116A11361224106E13501122C6512F
:1005C000146E156A10501424C36F06DE640EE66EB6
:1005D000E66AE66AE66A19DBE552E552E552E5525B
:1005E000D00EE66E90DDE5520101A46F31DD010110
:1005F000A66FC3C1E6FF87DDE5520101A46F28DDC8
:100600000101A66FD3DDE8DDD10EE66E7CDDE5529B
:100610000101A46F1DDD0101A66F40DD0F0B01017B
:10062000CD6F16DD0101A66F39DD0101CC6F10DD44
:100630000101A66F33DD0101CB6F0ADD0101A66F59
:100640002DDD0101A56FF2DCB1DD0101CE6BE552BC
:10065000E7CFD9FF1200948E949C400EAF6EAC8A07
:10066000AC84AC9CAB8EAB889E989D8AF28EF28C4B
:100670001200D9CFE6FFE1CFD9FFE6520101A05128
:100680009E1902E1A1519F1901E1F8D79EC1E9FF2E
:100690009FC1EAFF9E2B000E9F23EFCFDFFF920E3C
:1006A0009E5D010E9F5904E36A0E9E6F010E9F6FBF
:1006B000DF5000D0E552E552E7CFD9FF1200D9CF85
:1006C000E6FFE1CFD9FFACA2FED7FE0EDB50AD6E48
:1006D0009EA8FED7E552E7CFD9FF1200D9CFE6FF9B
:1006E000E1CFD9FF030EE126FD0EDBCFDEFFDBCF2E
:1006F000DDFFBFDFE76E020EE7CFDBFFFC0EDB5056
:10070000F36E020EDB50F35C0DE0FD0EDBCFE9FF74
:10071000DB2AFE0EDBCFEAFF01E3DB2A020EDBCF92
:10072000EFFFE7D7FD0EDBCFE9FFFE0EDBCFEAFFE1
:10073000EF6ADECF10F0DDCF11F010C0F3FF11C073
:10074000F4FF030EE15C03E200D0E16AE552E16EE2
:10075000E552E7CFD9FF1200D9CFE6FFE1CFD9FFAD
:10076000020EE126DE6ADD6AFD0EDBCFE9FFFE0E3A
:10077000DBCFEAFFEF5014E0FD0EDBCFE9FFFE0E0A
:10078000DBCFEAFFEF50E66E9ADFE552DF2A010E7B
:1007900001E3DB2AFD0EDB2AFE0E01E3DB2AE4D7B0
:1007A000010EF36EF46A020EE15C03E200D0E16A2E
:1007B000E552E16EE552E7CFD9FF1200DACFE4FF50
:1007C000E2CFDAFFE9CFE4FFEACFE4FFE652D9CF88
:1007D000E6FFE1CFD9FFE6529EAA16D0AE50DF6EFB
:1007E0000101A0C1E9FFA1C1EAFFA02B000EA123D6
:1007F000DFCFEFFF920EA05D010EA15904E36A0E58
:10080000A06F010EA16F9E9AE552E552E7CFD9FF86
:10081000E552E5CFEAFFE5CFE9FFE5CFDAFF1100CA
:10082000DACFE4FFE2CFDAFFE652F2940101932936
:10083000936F8078E552E5CFDAFF1100D9CFE6FF5C
:10084000E1CFD9FF040EE126819A819481888184C9
:100850008194818881848194FD0EDB50040B02E039
:10086000818801D0819881848194FD0EDB50020B38
:1008700002E0818801D0819881848194FD0EDB5053
:10088000010B02E0818801D0819881848194819854
:1008900081848194818481948184020EDB6A030EB9
:1008A000DB6ADE6A080EDD6ED9CFE9FFDACFEAFF38
:1008B000010ED880EE54000EED5428E2819481A6FA
:1008C00012D0020EDBCF12F0030EDBCF13F0DE509E
:1008D0001224106EDD501320116E020E10C0DBFFCB
:1008E000030E11C0DBFF8184020E106E116A10C06E
:1008F0000BF011C00CF0DECF06F0DDCF07F00BECF3
:100900000FF006C0DEFF07C0DDFFCED7818A020EE2
:10091000DBCF10F0030EDBCF11F010C0F3FF11C0DE
:10092000F4FF040EE15C03E200D0E16AE552E16EFF
:10093000E552E7CFD9FF1200D9CFE6FFE1CFD9FFCB
:10094000FE0EDB50A96EA69EA69CA680F40EE66E57
:10095000010EE66EE66AE66A58D9E552E552E552BE
:10096000E552A85000D0E552E7CFD9FF1200D9CF09
:10097000E6FFE1CFD9FFFE0EDB50A96EFD0EDB5086
:10098000A86EA69EA684550EA76EAA0EA76EA68276
:10099000A1A8FED7A198A694E552E7CFD9FF1200EF
:1009A000D9CFE6FFE1CFD9FFFB0EDBCFE9FFFC0E8D
:1009B000DBCFEAFFEF501AE0FB0EDBCFE9FFDB2ACB
:1009C000FC0EDBCFEAFF01E3DB2AEF50E66EFD0E03
:1009D000DBCF10F0DB2AFE0EDBCF11F001E3DB2AC8
:1009E0001050E66EC4DFE552E552DED7E552E7CFA0
:1009F000D9FF1200D9CFE6FFE1CFD9FF020EE126E1
:100A0000FD0EDBCFE6FF98DFE552DE6EDD6AD9CF63
:100A1000E9FFDACFEAFFEE50ED1001E11ED0DFCFA3
:100A2000E6FF4DDEE552FD0EDB2AFE0E01E3DB2A7A
:100A3000FD0EDBCF10F0FE0EDBCF11F0113404E21F
:100A40001050FF08000E115401E207D0D9CFE9FF82
:100A5000DACFEAFFEE50ED10D3E1980EE66E3A0ED3
:100A6000E66EE66AE66AD1D8E552E552E552E5520D
:100A7000020EE15C02E2E16AE552E16EE552E7CF87
:100A8000D9FF1200D9CFE6FFE1CFD9FF040EE1264E
:100A900001015A0E9C6F010E9D6F9CC1E6FF9DC126
:100AA000E6FFFD0EDBCFE6FFFE0EDBCFE6FF7BECC5
:100AB0000CF0E552E552E552E5529CC1E6FF9DC1BE
:100AC000E6FFD9EC0EF0E552E552F3CFDEFFF4CFAE
:100AD000DDFFD9CFE9FFDACFEAFF020EEECFDBFF71
:100AE000030EEDCFDBFF020EDBCF10F0030EDBCFEA
:100AF00011F0040E105C000E11580AE2300EE66E82
:100B0000DEDDE552020EDB2A030E01E3DB2AEBD722
:100B10009CC1E6FF9DC1E6FF1FDEE552E552F3CF23
:100B2000DEFFF4CFDDFF040EE15C02E2E16AE55294
:100B3000E16EE552E7CFD9FF1200D9CFE6FFE1CF52
:100B4000D9FFE652800EDF6EDF50000811E2FE0E84
:100B5000DB50DF1405E0310EE66EB1DDE55204D066
:100B6000300EE66EACDDE552DF407F0BDF6EECD77A
:100B7000E552E552E7CFD9FF1200D9CFE6FFE1CF2A
:100B8000D9FF020EE126FE0EDB50F00BE8380F0B0A
:100B9000300FDF6EDF50390803E2070EDF24DF6E0F
:100BA000FE0EDB500F0B300FE76E010EE7CFDBFFC1
:100BB000DB5039080AE2070E106E010EDBCFE7FFAB
:100BC0001050E726010EE7CFDBFFDFCFE6FF77DD32
:100BD000E552010EDBCFE6FF72DDE552680EE66EF0
:100BE0006EDDE552020EE15C02E2E16AE552E16E81
:100BF000E552E7CFD9FF12000D0EE66E60DDE5523B
:100C00000A0EE66E5CDDE5521200D9CFE6FFE1CFB9
:100C1000D9FFFB0EDBCF05F0FC0EDBCF06F0FD0E9F
:100C2000DBCF07F0FE0EDBCF08F00834000E08180B
:100C300009E6D880000E0554000E0654000E075435
:100C4000000E08540CE2D950FB0FE96EFF0EDA20BB
:100C5000EA6EEE06000EEE5AEE5AEE5ADAD7E5527A
:100C6000E7CFD9FF1200D9CFE6FFE1CFD9FF020EBF
:100C7000E126DE6ADD6ADECF10F0DDCF11F0FE0E78
:100C8000DB50000111AE02D0D89003D0105C000EF2
:100C9000115809E2200EE66E12DDE552DF2A010E40
:100CA00001E3DB2AE8D7020EE15C02E2E16AE552E9
:100CB000E16EE552E7CFD9FF12008168480E936ECE
:100CC000806A896A2F0E926E820EC16E010EC26E0C
:100CD0008268800E946E948E949C1200980EE66E3C
:100CE0003A0EE66EE66AE66A90DFE552E552E552B4
:100CF000E552E3DF8190808801016A0EA06F010E4A
:100D0000A16FA0C19EF1A1C19FF10101180E586F02
:100D1000010E596F01015A0E9C6F010E9D6F9BDCF5
:100D2000080EE66ECCDCE552100EE66E270EE66E7F
:100D3000E66AE66A6ADFE552E552E552E5525CDFB3
:100D400058C1E6FF59C1E6FF07DDE552E552F3CF92
:100D5000B1F1F4CFB2F150DF000EE66EE66A4ADE82
:100D6000E552E552600EE66EE66A44DEE552E55273
:100D7000800EE66EE66A3EDEE552E552A00EE66EB5
:100D8000E66A38DEE552E552C00EE66EE66A32DE0D
:100D9000E552E552E00EE66EE66A2CDEE552E552DB
:100DA0002BDF81808098100EE66E270EE66EE66AD5
:100DB000E66A2BDFE552E552E552E552400EE66E5B
:100DC0006EEC01F0E5520101A869A8C1E6FF400EF2
:100DD000E66EEFEC01F0E552E55202C110F003C1FE
:100DE00011F0126A10C0E6FF11C0E6FF12C0E6FF64
:100DF000180EE66E010EE66EC0EC0EF0136E050ED8
:100E0000E15E1350180EE66E010EE66EA5DCE552AB
:100E1000E552F3CFB1F1F4CFB2F1EEDE100EE66E93
:100E2000270EE66EE66AE66AF0DEE552E552E55226
:100E3000E5528BEC02F00EC110F00FC111F0126AF6
:100E400010C0E6FF11C0E6FF12C0E6FF180EE66E06
:100E5000010EE66EC0EC0EF0136E050EE15E13504F
:100E6000180EE66E010EE66E77DCE552E552F3CF22
:100E7000B1F1F4CFB2F1100EE66E270EE66EE66A1F
:100E8000E66AC3DEE552E552E552E552070EE66E2C
:100E9000A00EE66EE7EC0EF0E552E55210C110F040
:100EA00011C111F0126A10C0E6FF11C0E6FF12C0B6
:100EB000E6FF180EE66E010EE66EC0EC0EF0136E45
:100EC000050EE15E1350180EE66E010EE66E44DC70
:100ED000E552E552F3CFB1F1F4CFB2F18DDE100E51
:100EE000E66E270EE66EE66AE66A8FDEE552E552AA
:100EF000E552E5520101AF6BB06B0101070EAF5D2A
:100F0000000EB0593CE2AFC1E6FFB0C1E6FF96DC8F
:100F1000E552E552F3CF94F1F4CF95F1880EE66EE9
:100F2000130EE66EE66AE66A70DEE552E552E552B9
:100F3000E5524D0EE66E5FEC03F0E552300E010116
:100F4000AF25E66E5FEC03F0E5523D0EE66E5FEC1A
:100F500003F0E55294C1E6FF95C1E6FF93DDE5524B
:100F6000E552060EE66E5FEC03F0E552020EE66E09
:100F70007ADEE5520101AF2B000EB023BED7100E72
:100F8000E66E270EE66EE66AE66A3FDEE552E55259
:100F9000E552E55231DE0101AF6BB06B0101050E88
:100FA000AF5D000EB05948E2AFC1E6FF21EC0FF093
:100FB000E5520A0EE66E55EC0FF0E55269EC0FF0C3
:100FC00007EC00F0000901E0FBD760EC0FF0F3CF75
:100FD00094F1F4CF95F1410EE66E5FEC03F0E5522B
:100FE000300E0101AF25E66E5FEC03F0E5523D0ED9
:100FF000E66E5FEC03F0E55294C1E6FF95C1E6FFB3
:1010000041DDE552E552060EE66E5FEC03F0E55277
:10101000020EE66E28DEE552F40EE66E010EE66E76
:10102000E66AE66AF2DDE552E552E552E552010173
:10103000AF2B000EB023B2D7E80EE66E030EE66EBD
:10104000E66AE66AE2DDE552E552E552E552D4DDB4
:101050000101AD6BAE6B0101040EAD5D000EAE592A
:1010600075E2560EE66E5FEC03F0E552300E0101BC
:10107000AD25E66E5FEC03F0E5523D0EE66E5FECEB
:1010800003F0E552ADC1E6FFAEC1E6FFA2EC02F00F
:10109000E552E55258C1E6FF59C1E6FFCBC1E6FF74
:1010A000CCC1E6FFCDC1E6FFCEC1E6FF15EC0DF0E9
:1010B000106E060EE15E105058C1E6FF59C1E6FF02
:1010C000D9EC0EF0E552E552F3CFB1F1F4CFB2F125
:1010D0000101060ED880B157000EB2570101060E6D
:1010E000B15D000EB25911E20101000ED880B15578
:1010F000000EB2550AE2300EE66E5FEC03F0E552E8
:101100000101B107000EB25BEFD758C1E6FF59C12C
:10111000E6FFACEC03F0E552E552F3CFB1F1F4CFCA
:10112000B2F12C0EE66E5FEC03F0E552500EE66E67
:10113000C30EE66EE66AE66A68DDE552E552E55200
:10114000E5520101AD2B000EAE2385D7819080883A
:1011500053DD12C110F013C111F0126A10C0E6FF86
:1011600011C0E6FF12C0E6FF180EE66E010EE66E35
:10117000C0EC0EF0136E050EE15E1350180EE66E15
:10118000010EE66EACEC03F0E552E552F3CFB1F19F
:10119000F4CFB2F1100EE66E270EE66EE66AE66A4E
:1011A00034DDE552E552E552E5520101AD6BAE6B1F
:1011B0000101000EAD5D010EAE591EE20101AD2927
:1011C000E86C0101A86FA8C1E6FF400EE66EEFECE7
:1011D00001F0E552E5528170F40EE66E010EE66E06
:1011E000E66AE66A12DDE552E552E552E552010192
:1011F000AD2B000EAE23DCD7F00EE66E490EE66E88
:10120000020EE66EE66A01DDE552E552E552E55270
:1012100014C110F015C111F0126A10C0E6FF11C020
:10122000E6FF12C0E6FF180EE66E010EE66EC0EC99
:101230000EF0136E050EE15E1350180EE66E010EF1
:10124000E66EACEC03F0E552E552F3CFB1F1F4CF2A
:10125000B2F1100EE66E270EE66EE66AE66AD5DC9F
:10126000E552E552E552E552E668400EE66EEFECD7
:1012700001F0E552E5520101010EAC6F010E0101D2
:10128000AD6FAE6B0101090EAD5D000EAE591FE2F0
:101290000101AC29E86C0101A86FA8C1E6FF400E6E
:1012A000E66EEFEC01F0E552E5520101AC47880E25
:1012B000E66E130EE66EE66AE66AA7DCE552E552D4
:1012C000E552E5520101AD2B000EAE23DBD7A00E97
:1012D000E66E860EE66E010EE66EE66A96DCE55276
:1012E000E552E552E55216C110F017C111F0126A2D
:1012F00010C0E6FF11C0E6FF12C0E6FF180EE66E52
:10130000010EE66EC0EC0EF0136E050EE15E13509A
:10131000180EE66E010EE66EACEC03F0E552E552F7
:10132000F3CFB1F1F4CFB2F1100EE66E270EE66EF8
:10133000E66AE66A6ADCE552E552E552E5520101E9
:10134000800EAC6F010E0101AD6FAE6B0101090E95
:10135000AD5D000EAE591FE20101AC29E86C010140
:10136000A86FA8C1E6FF400EE66EEFEC01F0E55273
:10137000E5520101AC43880EE66E130EE66EE66A96
:10138000E66A43DCE552E552E552E5520101AD2B38
:10139000000EAE23DBD7A00EE66E860EE66E010EC3
:1013A000E66EE66A32DCE552E552E552E552E66861
:1013B000400EE66EEFEC01F0E552E55204C110F08C
:1013C00005C111F0126A10C0E6FF11C0E6FF12C09D
:1013D000E6FF180EE66E010EE66EC0EC0EF0136E20
:1013E000050EE15E1350180EE66E010EE66EACECD3
:1013F00003F0E552E552F3CFB1F1F4CFB2F106C1FB
:1014000010F007C111F0126A10C0E6FF11C0E6FF2C
:1014100012C0E6FF180EE66E010EE66EC0EC0EF08E
:10142000136E050EE15E1350180EE66E010EE66EA9
:10143000ACEC03F0E552E552F3CFB1F1F4CFB2F1E9
:10144000100EE66E270EE66EE66AE66A05EC06F01A
:10145000E552E552E552E5520101A96BAA6B010183
:10146000A05101019E1904E10101A15101019F193F
:1014700028E039EC03F00101A36F0101A351106EC4
:10148000116AFF0ED8801056000E115610C0A8F138
:10149000450EE66E5FEC03F0E5523D0EE66E5FEC46
:1014A00003F0E5520101A3510101946F956B94C1C2
:1014B000E6FF95C1E6FF42EC05F0E552E552FCEC93
:1014C00005F0230EE66E5FEC03F0E552A9C1E6FFDE
:1014D000AAC1E6FF42EC05F0E552E552090EE66EC0
:1014E0005FEC03F0E552880EE66E130EE66EE66AD8
:1014F000E66A05EC06F0E552E552E552E552000ECB
:10150000E66EE66AA2EC02F0E552E552CBC1B3F119
:10151000CCC1B4F1CDC1B5F1CEC1B6F1880EE66E45
:10152000130EE66EE66AE66A05EC06F0E552E55251
:10153000E552E552A8C1E6FF400EE66EEFEC01F081
:10154000E552E552D00EE66E070EE66EE66AE66AF2
:1015500005EC06F0E552E552E552E5524C0EE66E1A
:101560005FEC03F0E552140EE66E400EE66E1BECE7
:1015700002F0E552E5520101AC6F0101AC29E86CC3
:101580000101AB6FABC1E6FF9DEC05F0E5523B0EF0
:10159000E66E5FEC03F0E552D00EE66E070EE66EE7
:1015A000E66AE66A05EC06F0E552E552E552E552D8
:1015B000520EE66E5FEC03F0E552130EE66E400E3F
:1015C000E66E1BEC02F0E552E5520101A76F010146
:1015D000A729E86C0101AB6FABC1E6FF9DEC05F0FC
:1015E000E5523B0EE66E5FEC03F0E552010EE66E4F
:1015F000E66AA2EC02F0E552E552CBC1B7F1CCC1EC
:10160000B8F1CDC1B9F1CEC1BAF1880EE66E130EB4
:10161000E66EE66AE66A05EC06F0E552E552E5524A
:10162000E5520101AF6BB06B0101050EAF5D000E1D
:10163000B05946E2AFC1E6FF21EC0FF0E5520A0EC9
:10164000E66E55EC0FF0E55269EC0FF007EC00F098
:10165000000901E0FBD760EC0FF0F3CF94F1F4CF79
:1016600095F1410EE66E5FEC03F0E552300E01019C
:10167000AF25E66E5FEC03F0E5523D0EE66E5FECE3
:1016800003F0E552E80EE66E030EE66EE66AE66AE1
:1016900005EC06F0E552E552E552E55294C1E6FF4D
:1016A00095C1E6FF42EC05F0E552E5523B0EE66ED1
:1016B0005FEC03F0E5520101AF2B000EB023B4D76D
:1016C000020EE66EE66AA2EC02F0E552E552CBC1EC
:1016D000BBF1CCC1BCF1CDC1BDF1CEC1BEF1880E14
:1016E000E66E130EE66EE66AE66A05EC06F0E55273
:1016F000E552E552E5520101AF6BB06B0101080EF6
:10170000AF5D000EB0593BE2AFC1E6FFB0C1E6FFEE
:101710001EEC04F0E552E552F3CF94F1F4CF95F1CD
:101720004D0EE66E5FEC03F0E552300E0101AF2581
:10173000E66E5FEC03F0E5523D0EE66E5FEC03F003
:10174000E55294C1E6FF95C1E6FF42EC05F0E55293
:10175000E552D00EE66E070EE66EE66AE66A05EC26
:1017600006F0E552E552E552E5523B0EE66E5FECBF
:1017700003F0E5520101AF2B000EB023BFD7030EDB
:10178000E66EE66AA2EC02F0E552E552CBC1BFF18B
:10179000CCC1C0F1CDC1C1F1CEC1C2F1880EE66E9F
:1017A000130EE66EE66AE66A05EC06F0E552E552CF
:1017B000E552E5520101AF6BB06B0101040EAF5D64
:1017C000000EB05901E382D0560EE66E5FEC03F0D6
:1017D000E552300E0101AF25E66E5FEC03F0E552F5
:1017E0003D0EE66E5FEC03F0E55258C1E6FF59C1CD
:1017F000E6FFAFC1E9FFB0C1EAFF020ED890E936BB
:10180000EA36E806FBE1B30EE926010EEA22EECF46
:10181000E6FFEECFE6FFEECFE6FFEFCFE6FF15ECFB
:101820000DF0106E060EE15E105058C1E6FF59C172
:10183000E6FFD9EC0EF0E552E552F3CFB1F1F4CF6B
:10184000B2F10101060ED880B157000EB257010166
:10185000060EB15D000EB25911E20101000ED880F2
:10186000B155000EB2550AE2300EE66E5FEC03F0A1
:10187000E5520101B107000EB25BEFD758C1E6FF98
:1018800059C1E6FFACEC03F0E552E552F3CFB1F1FC
:10189000F4CFB2F1E80EE66E030EE66EE66AE66A93
:1018A00005EC06F0E552E552E552E5520101030E62
:1018B000AF5D000EB05905E23B0EE66E5FEC03F043
:1018C000E5520101AF2B000EB02377D70101A92B00
:1018D000000EAA23FCEC05F0980EE66E3A0EE66EBA
:1018E000E66AE66A05EC06F0E552E552E552E55295
:0618F0008170B5D5120065
:0A18F600D9CFE6FFDACFE6FFFA0EC5
:10190000E3CFD9FFFB0EE3CFDAFFFD0EE35209E789
:101910002D0EDE6EFC0EE31EE32AFD0ED8B4E306A8
:10192000E31EE652E652E652FD0EE124E76EFF0E9C
:10193000E220E46EE652F70EE3CFE6FFF70EE3CFC8
:10194000E6FFEBEC0CF0F90EE124E96EFF0EE2206D
:10195000EA6EDBEC0CF00AE1D8EC0CF009E1DBEC10
:101960000CF008E1D8EC0CF007E108D0E6EC0CF044
:10197000E1EC0CF0E6EC0CF0E1EC0CF0E6EC0CF039
:10198000DE6AF90EE126FF0EE222FF0EE3CFDAFF58
:10199000E552FF0EE3CFD9FFE552FC0EE124E96EDC
:1019A000FF0EE220EA6EEECFF3FFEFCFF4FF12005E
:1019B000EF380F0B1200EF500F0B02E1EE52D884FC
:1019C0001200EF380F0B300FDE6E1200EE500F0BCF
:1019D000300FDE6E1200FC0EE3CFE9FFFD0EE3CF09
:1019E000EAFF100EE66EEE6AEE6AEF6AD890FD0E20
:1019F000E336FE0EE336ED36ED36EF36FF0EE30648
:101A000009E00CEC0DF0EE520CEC0DF0EE520CEC8B
:101A10000DF0EDD7E56E1200030EEF24E8B6EF6E81
:101A2000300EEF24E8BEEF6E000CD9CFE6FFDACF20
:101A3000E6FFF80EE3CFD9FFF90EE3CFDAFFE65267
:101A4000E652E652E652E652FB0EE124E76EFF0E46
:101A5000E220E46EE652F30EE3CFE6FFF30EE3CFAF
:101A6000E6FFF30EE3CFE6FFF30EE3CFE6FF9AECDB
:101A70000DF0F50EE124E96EFF0EE220EA6E87EC30
:101A80000DF019E18AEC0DF018E187EC0DF017E18B
:101A90008AEC0DF016E187EC0DF015E18AEC0DF003
:101AA00014E187EC0DF013E18AEC0DF012E187EC04
:101AB0000DF011E112D090EC0DF095EC0DF090ECE2
:101AC0000DF095EC0DF090EC0DF095EC0DF090EC28
:101AD0000DF095EC0DF090EC0DF095EC0DF0DE6A4C
:101AE000F50EE126FF0EE222FF0EE3CFDAFFE5520C
:101AF000FF0EE3CFD9FFE552FA0EE124E96EFF0EA7
:101B0000E220EA6EEECFF3FFEFCFF4FF1200EF38E2
:101B10000F0B1200EF500F0B02E1EE52D8841200AF
:101B2000EF380F0B300FDE6E1200EE500F0B300F40
:101B3000DE6E1200FA0EE3CFE9FFFB0EE3CFEAFF01
:101B4000200EE66EEE6AEE6AEE6AEE6AEF6AD890F2
:101B5000FB0EE336FC0EE336FD0EE336FE0EE336F7
:101B6000ED36ED36ED36ED36EF36FF0EE3060FE0DF
:101B7000C9EC0DF0EE52C9EC0DF0EE52C9EC0DF0CF
:101B8000EE52C9EC0DF0EE52C9EC0DF0E1D7E56E66
:101B90001200030EEF24E8B6EF6E300EEF24E8BE1D
:041BA000EF6E000CD8
:0C1BA400506F727420636F6D6D20393635
:101BB0003030206F757665727400496E6974204903
:101BC000324320536F66742070696E733A20323747
:101BD0002D3E20534441202D3E203133202C2032F5
:101BE000382D3E2053434C202D3E203132004553AA
:101BF0004320706F757220736F727469720D00529A
:101C0000656375202009416374696F6E7320200934
:101C1000536F7274696573202009456E747265652F
:101C2000732020094144433130202009414443318D
:101C30003220202020202041444331380D00536FB2
:101C400072746965204E6F726D616C6520646520E9
:101C5000507267006361722072656375203A0049B3
:101C60006E6974204D4350323330313720457870DF
:101C7000616E64657220452F53200D00496E6974B2
:101C800020414443313862204D43503334323420B4
:101C90004932430D00496E6974204144433130623A
:101CA000205049433138460D00436C69676E6F74AC
:101CB000656D656E7420646573204C4544530D005A
:101CC0004D6F6E74656520312D3E203132380D0028
:101CD00044657363656E7465203132382D3E310D75
:011CE0000003
:0E1CE2001E0EF66E000EF76E000EF86E01017B
:101CF0000900F550D46F0900F550D56F03E1D467A2
:101D000001D03DD00900F550CF6F0900F550D06FDC
:101D10000900F550D16F09000900F550E96E09007E
:101D2000F550EA6E090009000900F550D26F09006C
:101D3000F550D36F09000900F6CFD6F1F7CFD7F1F0
:101D4000F8CFD8F1CFC1F6FFD0C1F7FFD1C1F8FF6E
:101D50000101D25302E1D35307E00900F550EE6EC2
:101D6000D207F8E2D307F9D7D6C1F6FFD7C1F7FFFC
:101D7000D8C1F8FF0101D407000ED55BBFD7120010
:101D8000FB0EE3CFF6FFFC0EE3CFF7FFFD0EE3CF34
:101D9000F8FFFE0EE3CFE9FFFF0EE3CFEAFFE9CF46
:101DA000F3FFEACFF4FF0900F5CFEFFFEE66FBD7B4
:101DB0001200FE0EE3CFE9FFFF0EE3CFEAFFF36A66
:0E1DC000F46AEE5203E0F34AF42AFBD7120055
:021DCE00D9CF6B
:101DD000E6FFDACFE6FFE1CFD9FFE2CFDAFFC26A52
:101DE000FD0EDB50C16EFC0EDB50380B106EFD0E8D
:101DF000DB50040DF350C00B1010C26EFC0EDBAEB6
:101E000003D09E9C9D8CF28CC280E552E5CFDAFF18
:061E1000E7CFD9FF12002C
:0A1E1600036A026A100EE76ED8900E
:101E200006360736023603360B50025C0C50035858
:101E300005E30B50025E0C50035A062AE72EF0D73A
:021E400012008E
:0E1E4200D9CFE6FFDACFE6FFE1CFD9FFE2CF3E
:101E5000DAFFC70EC214106EFD0EDB50380B1010E7
:0E1E6000C26EE552E5CFDAFFE7CFD9FF1200E0
:021E6E00000E64
:101E7000F36E00EE00F0060E01D81200EA6002D008
:0E1E8000EE6AFCD7F350E9601200EE6AFCD760
:021E8E0015EE4F
:101E900000F025EE00F0F86A0F9C71EC0EF06BEC90
:0A1EA0000FF06EEC06F0FBD7120005
:061EAA00FF0EE350E84EBC
:101EB0001200000000D000D000D0E82EFAD71200A7
:101EC000C450136E126AC3501210F36E13C0F4FFA5
:021ED0001200FE
:041ED200C2841200B4
:021ED6001200F8
:081ED800A41BBA1BEE1BFF1B4B
:101EE0003E1C541C5F1C7C1C951CA91CC01CD01CD7
:101EF0004331383A204D435032333031375F33333A
:101F000030345F333432345F4932435F736F667409
:101F10005F303331395F58706F72742E6300000088
:101F200000000000000000000000000000000000B1
:101F300018013132333435363738393031323334B1
:101F40003500313233343536373839303132333485
:101F50003536000000000000000000000000000016
:101F60000000000000000000000000000000000071
:021F700000006F
:020000040030CA
:01000300FEFE
:0200000400F00A
:10000000506F727420436F6D20313932303062206E
:100010002620496E69742049324320486172640089
:1000200056616C65757220536F7274696573203FF9
:1000300020203C4553433E206578697420202000F1
:10004000536F727469657320456E747265652041E3
:10005000444331302E2E2E2031322E2E31382000C6
:1000600055736167652049326320536F6674776109
:100070007265204D504C41422043313820200D0004
:10008000313846323532206176656320626F6F7495
:100090006C6F6164657220202020202020200D00DC
:1000A0007061756C666A756A6F40667265652E660A
:1000B00072202020202020202020202020200D0021
:1000C0004D504C4142204944452056382E36332E5F
:1000D0002E2E2E2E2E2E2E2E2E2E2E2E2E200D009D
:1000E0004D504C4142204331382076332E33372E49
:1000F0003031202E2E2E2E2E2E2E2E2E0D0A0000CA
:00000001FF
